:020000040000FA
:0A0000008316FF2390008312BB2833
:100100008101AF0A2F088207000087288728AF01E6
:1001100089289B2800000000011B802800000000A7
:1001200000000000000000000000000000000000CF
:10013000000000000000AB0125088207592A6C2A44
:10014000772A822A8D2A822A8D2A822A8D2A822A39
:100150008D2A822A8D2A822A8D2A822A8D2A822A13
:100160009B2AA92AB42ABF2ACA2AD52AE02AF02A19
:10017000FB2A0A2B152B0030B8008F23B900003062
:10018000850083160C308500831239088500013004
:10019000B8008F23AC00AC0DAC0DAC0D2C0D70393C
:1001A000703A8838B4000330B8008F23AC00AC0D2F
:1001B000AC0DAC0D2C0D7039703A8838B500053097
:1001C000B8008F23AC00AC0DAC0DAC0D2C0D70390C
:1001D000703A8838B6000730B8008F23AC00AC0DF9
:1001E000AC0DAC0D2C0D7039703A8838B700023068
:1001F000B8008F23033EAC002C0D0639B404AC0CC0
:100200002C0C3F398038B0000430B8008F23033EF7
:10021000AC002C0D0639B504AC0C2C0C3F398038E1
:10022000B1000630B8008F23033EAC002C0D063918
:10023000B604AC0C2C0C3F398038B2000830B80042
:100240008F23033EAC002C0D0639B704AC0C2C0CEC
:100250003F398038B300073084001130A400AE016C
:10026000A501A301A601A701A801A901AA01AF0147
:0C027000C530831681008312302A003450
:100460008A20851D3E2AAB1FAB0A20100310FC30EA
:100470002B07031C201400000000312A8A20851954
:10048000302AAB1FAB0A20100310FC302B07031CD3
:100490002014000000003F2A1130A400A501A30190
:1004A000A601A701A801A901AA01AB01F030A0058E
:1004B0000034000000000000201C672AA40B642AFE
:1004C0001130A400A50A00340000000000341130EF
:1004D000A400000000000034AE0B6F2ABB2800000F
:1004E0000000000000002018762AA50A0034000051
:1004F00000000000000000000000000020184C2A4E
:10050000A50A0034A50A031020180314AA0D000040
:1005100000000000000000000034000000000000A7
:100520000000A50A201C982A2A1C4C2A000000342E
:100530002A184C2A0034A30A2308A507000000004B
:10054000201CA62A2A1C4C2A000000342A184C2AF7
:10055000003420184C2AA50AA30A0000000000005D
:10056000000000000000003420184C2A2A08A600D1
:100570000330A50000000000000000000034201837
:100580004C2AA50AA30A0000000000000000000099
:100590000000003420184C2A2A08A7000330A500C8
:1005A00000000000000000000034A50AA30A0000BB
:1005B0000000000000000000000000000000003407
:1005C0002A08A8002018EB2A0330A500000000002C
:1005D000000000000034A501A301A901AA01292BF4
:1005E000A50AA30A000000000000000000000000AF
:1005F0000000000000342A08A9002018062B033050
:10060000A50000000000000000000034A501A301C7
:10061000AA01292B201C4C2AA50AA30A00000000CD
:1006200000000000000000000034201C4C2AA5013E
:10063000A301A0102013260803191F2B302920170F
:10064000212BAC01A601A701A801A901AA01A301C0
:10065000302AFF3A26082706280629062A06031DFF
:10066000212BAE01A71F792B3908AC0034082706CF
:10067000FE390319552335082706FE3903195E2371
:1006800036082706FE390319672337082706FE397F
:100690000319702339082C060319212B390885000A
:1006A0000030B80039089623212B30082606031D98
:1006B000080027183914271C3910080031082606AD
:1006C000031D08002718B914271CB91008003208A8
:1006D0002606031D080027183916271C39120800A2
:1006E00033082606031D08002718B916271CB9125F
:1006F000080027080A3A0F39031D212B2808031D7B
:10070000212B270835067039031D212B0230B80034
:100710002908962383169C188B2B831230293808BE
:1007200083169B001C141A088312080083169A0073
:1007300083123808013C031C0800380883169B000C
:100740001C1555309D00AA309D009C148312080092
:0407F8008312BB2885
:02400E00C431BB
:1042000003000100010001000200010003000100A1
:024210000400A8
:00000001FF
